:100000000C308A00B22C0000D422532AA0264F2A9A
:100010004F29D5060A00CC22D62CA0264F2A4F29DC
:1000200020224F28D222C42A0D050001D22C4324BD
:10003000CC27532A3A10A53A0D050000D22C4324B0
:10004000CC27532A3A10A53A0D050001CC22D62C14
:10005000A0264F2A4F2920224F2D4122D5060A00E3
:10006000D22C4324CC27532A3A10A53A0D0500017F
:10007000D22C4324CC27532A3A10A53A0D0500016F
:100080005029412B5910CD27D4275210C42750296D
:100090004522D5060A00D22C4324CC27532A3A10F5
:1000A000A53A0D050001D22C4324CC27532A3A103F
:1000B000A53A0D0500015029412B5910CD27D42711
:1000C0005210C427DA20C42A0D050001D22C432483
:1000D000CC27532A3A10A53A0D050001D22C43240F
:1000E000CC27532A3A10A53A0D050001CB27CE2282
:1000F0004310D422532A5510CD27D427D22A0D05D8
:100100000000CC22D6203A10A53AA00400015029C4
:10011000412B411DA0127510090053244129501D87
:10012000A01275100900D027CC27C8203A10A53A94
:100130000900CC2FCE20D2205A1DA0127510090024
:10014000D02FCE20D2205A1DA01275100D0500010F
:10015000CC32F63C20376139613DEE346B102D1006
:10016000F432733AA027CC29C1060A005039613B0A
:100170007910EE30F2307A37E935A016203AE539B9
:100180007410ED37F437F23A0D050001D422532AEA
:10019000A027CC29C1060A00633A6537E9060A00A0
:1001A000D027D72252104F27A0060A00CF252110B2
:1001B0000D050001D62C4229412AA0264F222E17D8
:1001C0002E100D0500008316861383128613083047
:1001D000F800EA280000F817FF28F8138316031721
:1001E000CB0C8312031303188617031C861378178E
:1001F000FF287813F80BEE28FD28000086173F3003
:100200008400840B01290000F81BED28781BF928D5
:100210000800831603178C170C14000000008312CB
:100220000C087F39031955298316C70083120D085E
:100230008316C80083120F088316C9004708CB0035
:1002400083120313E32083160317480883128D00DB
:100250008316490883128F0083168C170C14000034
:10026000000083120C0D0E0D7F39031955298316DA
:10027000C70083120D088316C80083120F08831667
:10028000C9004708CB0083120313E320831603172A
:10029000480883128D008316490883128F008D0A47
:1002A00003198F0A03130929031703130800831680
:1002B00008108312081083168810831288109B017F
:1002C00008008316081183120811831688118312FF
:1002D00088119501080083160317CA014A084902CC
:1002E000031C7E2903138812831288168316881232
:1002F0008312881283160317CA0A6E298312031306
:1003000008008316881283128816831688128312B7
:10031000881208008316081283120812812183169E
:100320000317CC01CB01CC08031DB6294B08073CB1
:10033000031CB62949084B07840083134A18831706
:100340000008CD004D0BAB290313081283120816C9
:10035000AF29831603170313081283120812812191
:1003600083160317CB0A0319CC0A93290313081227
:1003700083120816812108008316081283120812BE
:1003800083168812831288121E3083160317C90041
:10039000831203136B2183160812831208160A3086
:1003A00083160317C900831203136B2183160317E7
:1003B000CA012930C900831203138A21053083162C
:1003C0000317C900831203136B2183160317CA0195
:1003D0003130C900831203138A2183160317CA011F
:1003E0003930C900831203138A218A150A120F2E8D
:1003F00083160317CA014130C900831203138A21EF
:1004000083160317CA015930C900831203138A21C6
:1004100083160317CA016130C900831203138A21AE
:1004200083160317CA01A830C900831203138A2157
:1004300083160317CA014930C900831203138A21A6
:1004400083160317CA015930C900831203138A2186
:1004500083160317CA016930C900831203138A2166
:1004600083160317CA01A830C900831203138A2117
:1004700083160317CA015130C900831203138A215E
:1004800083160317CA015930C900831203138A2146
:1004900083160317CA01A030C900831203138A21EF
:1004A00083160317CA01A830C900831203138A21D7
:1004B0008A150A12122E083083160317CE02031C67
:1004C0006D2ACE30840083170310800C00080319B6
:1004D0006D2A6B2A0000800B6A2A8312031308001E
:1004E000831603174A08CC004908CB00CB08031D2C
:1004F0007C2ACC080319BD2A0313061283120616A0
:100500008316861283128612831603174808CD00BD
:10051000CD0ACD030319942AFF30CE0083120313B2
:100520005B2283160317892A4708CE008312031320
:100530005B22831686128312861683160612831296
:100540000612831603174808CD00CD0ACD03031900
:10055000B12AFF30CE00831203135B2283160317E8
:10056000A62A4708CE00831203135B2283160317C3
:100570004B080319CC03CB03762A8312031308001C
:10058000C8308400831700080319D32A0230F8000A
:10059000F701F70BC92AF80BC82A9730F700F70BB9
:1005A000CF2A800BC62A08000030F8001F08C33984
:1005B00078049F000630F700F70BDC2A00009F1438
:1005C0009F18E02A1E08FD000430F8001F08C339F8
:1005D00078049F000630F700F70BEC2A00009F1408
:1005E0009F18F02A1E08FE0008000830F8001F08B7
:1005F000C33978049F000630F700F70BFD2A00008E
:100600009F149F18012B1E088316C900831208002F
:1006100083160317C601F201F101F401F301CA01C7
:10062000B030C900831203138A21163083160317D2
:10063000C900831203136B2183160317CA01B83054
:10064000C900831203138A21053083160317C900DA
:10065000831203136B2183160317CA01C030C9002C
:10066000831203138A218316CC164C088700831249
:10067000871A782B83160317C801C7014708073C60
:10068000031C582B8312031381218316CC164C08AC
:1006900087008312871E522B831603174814502B92
:1006A00083120313031083160317C80DC70A3E2BCA
:1006B000831203138121831603174608333C031C5E
:1006C0006B2B103071078400831748088000F10AF3
:1006D0000319F20A742B90307307840083174808BB
:1006E0008000F30A0319F40AC60A7B2B8312031352
:1006F0008121831603174608653C031C822B831255
:100700000313332B831203130800F5018316031719
:10071000C6014608333C031CA52B10304607840055
:1007200083170008C7004708103C031D992BC80A0F
:100730009A2BC8014808043C0318A32B4608F5006F
:100740007B103730C600C60A892BC6014608333CE9
:10075000031CC32B90304607840083170008C70092
:100760004708103C031DB62BC80AB72BC801480820
:10077000043C0318C12B32304607F5007B14373098
:10078000C600C60AA62B831203130800831603179C
:100790008C170C14000000000318F12B83120C08B6
:1007A0007F398316C80083120D088316C90083128F
:1007B0000F088316CA004808CB0083120313E320F6
:1007C00083160317490883128D0083164A08831283
:1007D0008F0083168C170C1400000000C70BF12B40
:1007E000142C83120C0D0E0D7F398316C800831252
:1007F0000D088316C90083120F088316CA00480823
:10080000CB0083120313E3208316031749088312D6
:100810008D0083164A0883128F008D0A03198F0AF0
:1008200003108316C70BC82B83120313080083160B
:1008300003174A08F80149020318212C4908F70058
:100840002D2CF7010830CB00C90DF70D4A087702AF
:100850000318F700F80DCB0B242C831203130800A8
:100860007808831603174708C9006430CA0083124A
:1008700003131724770883160317C700780830304E
:10088000031D492CC81C542CC819542C481A20305C
:100890004C2CC81148124814F8077808CB00831272
:1008A0000313E320831603174708C9000A30CA0060
:1008B000831203131724770883160317C7007808D9
:1008C0003030031D692CC819712C481C712C481A32
:1008D0002030F8077808CB0083120313E320831637
:1008E00003173030C7074708CB0083120313E320F8
:1008F00008008316081083120814831688108312C8
:100900008810831603174708831203139B000800FF
:100910008316881083128814831608108312081017
:10092000831603174708831203139B0008008316DE
:1009300008118312081583168811831288118316F3
:1009400003174708831203139500080083168811C4
:100950008312881583160811831208118316031752
:100960004708831203139500080083160317C71B5B
:10097000CD2C0F30F700460EF7050A30770203182A
:10098000C42C3030F707C62C4708F7077708CB0090
:1009900083120313E320831603170F30C6050A30B2
:1009A00046020318D52C3030D72CC7134708C6078A
:1009B0004608CB0083120313E32008002208A1009D
:1009C0002308A2002408A3002508A4007508313CD0
:1009D000031CEE2C7508323CA500F12C3230750258
:1009E000A5002208210723072407250783160317DC
:1009F000C400C9000530CA00831203131724780805
:100A0000A6008A150A12CC2EF701F80183160317E7
:100A1000470803104818F707F70CF80CC818F70731
:100A2000F70CF80C4819F707F70CF80CC819F7077A
:100A3000F70CF80C481AF707F70CF80CC81AF70768
:100A4000F70CF80C481BF707F70CF80CC81BF70756
:100A5000F70CF80C8312031308000310250D8316FE
:100A60000317C30083120313260883160317C90054
:100A70006430CA00831203131724780883160317FF
:100A8000C6002D30C7004608C80083120313042592
:100A9000780883160317C400750876020318692DB9
:100AA00076087502C700C9006430CA0083120313B8
:100AB0001724780883160317C6001430C7004608A9
:100AC000C800831203130425780883160317C50092
:100AD000812D75087602C700C9006430CA008312F0
:100AE00003131724780883160317C6001430C700B1
:100AF0004608C800831203130425780883160317D9
:100B0000C50044084307450783120313A0008A1554
:100B10000A12CF2EFF3083160317C7008312031368
:100B20008824FF3083160317C7008312031397240A
:100B3000023083160317C300FA30C8008312031370
:100B4000C02283160317C30B9C2DFF30C7008312EE
:100B500003137924043083160317C300FA30C80046
:100B600083120313C02283160317C30BAE2DFF306D
:100B7000C70083120313A624023083160317C30091
:100B8000E130C80083120313C02283160317C30B7E
:100B9000C02DFF30C700831203139724063083163D
:100BA0000317C300FA30C80083120313C022831650
:100BB0000317C30BD22DFF30C70083120313A624E3
:100BC000023083160317C300E130C80083120313F9
:100BD000C02283160317C30BE42DFF30C700831216
:100BE00003139724023083160317C300FA30C8009A
:100BF00083120313C02283160317C30BF62D0313AE
:080C000083128A150A122E2F3F
:101000008A11D4228A158A11F5228A158A11082399
:101010008A158A1185238A15813003178D000030C7
:101020008F00031006308316C7008A118312031342
:10103000C6238A157D0883160317C7001B30C80016
:101040008A118312031330248A1520308316031764
:10105000CB008A1183120313E3208A15093083160B
:101060000317CB008A1183120313E3208A158730FC
:1010700003178D0000308F00031007308316C70060
:101080008A1183120313C6238A157E088316031759
:10109000C7001B30C8008A118312031330248A153D
:1010A000203083160317CB008A1183120313E32029
:1010B0008A15093083160317CB008A118312031394
:1010C000E3208A158D3003178D0000308F00031048
:1010D00007308316C7008A1183120313C6238A15AB
:1010E000831649080317C7001B30C8008A118312F2
:1010F000031330248A15203083160317CB008A117E
:1011000083120313E3208A15093083160317CB00DB
:101110008A1183120313E3208A15933003178D007D
:1011200000308F00031008308316C7008A11831225
:101130000313C6238A15750883160317C7001B30CF
:10114000C8008A118312031330248A1509308316CC
:101150000317CB008A1183120313E3208A15831629
:10116000081700308312081B013083160317C600CE
:10117000993083128D0000308F00031009308316E0
:10118000C7008A1183120313C6238A158316031717
:101190004608C7001B30C8008A118312031330248D
:1011A0008A15203083160317CB008A11831203138C
:1011B000E3208A15093083160317CB008A118312A6
:1011C0000313E3208A158316881700308312881BC7
:1011D000013083160317C600A03083128D00003043
:1011E0008F00031009308316C7008A11831203137E
:1011F000C6238A15831603174608C7001B30C8008C
:101200008A118312031330248A15203083160317A2
:10121000CB008A1183120313E3208A150D30831645
:101220000317CB008A1183120313E3208A150A30B7
:1012300083160317CB008A1183120313E3208A1548
:10124000831608178312081FAF2C83168817831282
:10125000881FAF2C83160317C8016430C700033002
:10126000CA00E830C9008A118312031370228A155C
:10127000A83003178D0000308F008A110313092155
:101280008A15B63003178D0000308F008A110313C2
:1012900009218A15023083160317C600FA30C800E8
:1012A0008A1183120313C0228A1583160317C60BF3
:1012B0004E29031388178312881F2F2C83160317B8
:1012C000C8016430C7000130CA00F430C9008A1177
:1012D0008312031370228A1583160317C801643022
:1012E000C700CA01C830C9008A11831203137022D3
:1012F0008A15043003178D0000308F008A11031304
:1013000009218A15043083160317C700FA30C80074
:101310008A1183120313C0228A1583160317C70B81
:1013200086290B3083128D0000308F008A11031341
:1013300009218A15043083160317C700FA30C80044
:101340008A1183120313C0228A1583160317C70B51
:101350009E29C601460FAD29EC294608C7008A110F
:101360008312031379248A15163003178D00003079
:101370008F0003100A308316C7008A1183120313EB
:10138000C6238A15831603174608C7001B30C800FA
:101390008A118312031330248A150D308316031724
:1013A000CB008A1183120313E3208A150A308316B7
:1013B0000317CB008A1183120313E3208A1505302B
:1013C00083160317C8008A1183120313C0228A15DB
:1013D00083160317C60AAA29FF30C600C6080319D8
:1013E000302A4608C7008A118312031379248A150C
:1013F0001E3003178D0000308F0003100A30831653
:10140000C7008A1183120313C6238A158316031794
:101410004608C7001B30C8008A118312031330240A
:101420008A150D3083160317CB008A11831203131C
:10143000E3208A150A3083160317CB008A11831222
:101440000313E3208A15053083160317C8008A1199
:1014500083120313C0228A1583160317C603EE29CD
:10146000263083128D0000308F008A11031309216A
:101470008A15043083160317C700FA30C8008A1192
:1014800083120313C0228A1583160317C70B3D2A44
:10149000C601460F4C2A8B2A4608C7008A118312C0
:1014A000031388248A15303003178D0000308F0015
:1014B00003100A308316C7008A1183120313C62350
:1014C0008A15831603174608C7001B30C8008A1107
:1014D0008312031330248A150D3083160317CB00B3
:1014E0008A1183120313E3208A150A308316031727
:1014F000CB008A1183120313E3208A15053083166B
:101500000317C8008A1183120313C0228A15831699
:101510000317C60A492AFF30C600C6080319CF2A96
:101520004608C7008A118312031388248A153830AD
:1015300003178D0000308F0003100A308316C70098
:101540008A1183120313C6238A15831603174608CC
:10155000C7001B30C8008A118312031330248A1578
:101560000D3083160317CB008A1183120313E32077
:101570008A150A3083160317CB008A1183120313CE
:10158000E3208A15053083160317C8008A118312D9
:101590000313C0228A1583160317C6038D2A403011
:1015A00083128D0000308F008A11031309218A15E0
:1015B000043083160317C700FA30C8008A1183125B
:1015C0000313C0228A1583160317C70BDC2AC60132
:1015D000460FEB2A2A2B4608C7008A1183120313F1
:1015E00097248A154B3003178D0000308F000310AD
:1015F0000A308316C7008A1183120313C6238A1583
:10160000831603174608C7001B30C8008A118312CF
:10161000031330248A150D3083160317CB008A116B
:1016200083120313E3208A150A3083160317CB00B5
:101630008A1183120313E3208A15053083160317DA
:10164000C8008A1183120313C0228A158316031758
:10165000C60AE82AFF30C600C60803196E2B4608E2
:10166000C7008A118312031397248A155330031776
:101670008D0000308F0003100A308316C7008A11D6
:1016800083120313C6238A15831603174608C7005F
:101690001B30C8008A118312031330248A150D30C1
:1016A00083160317CB008A1183120313E3208A15D4
:1016B0000A3083160317CB008A1183120313E32029
:1016C0008A15053083160317C8008A118312031385
:1016D000C0228A1583160317C6032C2B5B30831296
:1016E0008D0000308F008A11031309218A15043000
:1016F00083160317C700FA30C8008A118312031338
:10170000C0228A1583160317C70B7B2BC601460F11
:101710008A2BC92B4608C7008A1183120313A624FB
:101720008A15663003178D0000308F0003100A30D1
:101730008316C7008A1183120313C6238A158316E2
:1017400003174608C7001B30C8008A118312031311
:1017500030248A150D3083160317CB008A118312AB
:101760000313E3208A150A3083160317CB008A116E
:1017700083120313E3208A15053083160317C8006C
:101780008A1183120313C0228A1583160317C60A0F
:10179000872BFF30C600C60803190D2C4608C7006A
:1017A0008A1183120313A6248A156E3003178D0045
:1017B00000308F0003100A308316C7008A1183128D
:1017C0000313C6238A15831603174608C7001B3068
:1017D000C8008A118312031330248A150D30831632
:1017E0000317CB008A1183120313E3208A150A30F2
:1017F00083160317CB008A1183120313E3208A1583
:10180000053083160317C8008A1183120313C02200
:101810008A1583160317C603CB2B8A118312031371
:1018200057218A158A1161218A15763003178D0098
:1018300000308F008A11031309218A1504308316A2
:101840000317C700FA30C8008A1183120313C0229D
:101850008A1583160317C70B222C831203138316D2
:1018600008178312081FAA2C83160317C8016430B7
:10187000C7000130CA00F430C9008A118312031373
:1018800070228A15C63003178D0000308F008A1130
:10189000031309218A158A1108238A15CC300317EE
:1018A0008D0000308F008A11031309218A158316D9
:1018B0000317C501C401C508031D802C4408333C2F
:1018C000031C802C10304407840083170008C300D9
:1018D0004308C6005730C7008A1183120313B5248A
:1018E0008A15203083160317CB008A118312031345
:1018F000E3208A1583160317C40A0319C50A5B2C53
:10190000C501C401C508031DA72C4408333C031CB2
:10191000A72C90304407840083170008C3004308B5
:10192000C6005730C7008A1183120313B5248A15E5
:10193000203083160317CB008A1183120313E32090
:101940008A1583160317C40A0319C50A822C831249
:1019500003134B2C831603175929831203138A157B
:101960000A12872E840183131F308305713083167A
:101970008F000F0886138312861783160317090832
:10198000C039890003131F129F120030031788000B
:10199000831287018801890101300313A900AA007D
:1019A000AB01AC00AD00AE01AF01B001B100B200BF
:1019B000B300B400B500B601B700B801B901BA016F
:1019C000BB01BC01BD01BE01BF01C001C101C2011B
:1019D000C301C401C501C601C700C801C901CA00CD
:1019E000CB01CC01CD01CE01CF00D001D101D2017C
:1019F000D300D401D501D601D700D801D900DA012E
:101A0000DB01DC01DD01DE01DF01E000E100E201DC
:101A1000E301E401E501E601E700E801E900EA008D
:101A2000EB01EC01ED01EE01EF00F0018316A000E7
:101A3000A101A200A301A401A501A600A701A8007D
:101A4000A901AA00AB01AC01AD01AE01AF01B0012B
:101A5000B101B201B300B401B501B601B701B801DB
:101A6000B901BA01BB01BC00BD01BE01BF01C0018B
:101A7000C100C201C301C401C501C601C70183126F
:101A80000317900191019201930194019501960130
:101A90009701980199019A019B019C019D019E016A
:101AA0009F01A001A101A201A301A401A501A6011A
:101AB000A701A801A901AA01AB01AC01AD01AE01CA
:101AC000AF01B001B101B201B301B401B501B6017A
:101AD000B701B801B901BA01BB01BC01BD01BE012A
:101AE000BF01C001C101C2018316900191019201A1
:101AF00093019401950196019701980199019A012A
:101B00009B019C019D019E019F01A001A101A201D9
:101B1000A301A401A501A601A701A801A901AA0189
:101B2000AB01AC01AD01AE01AF01B001B101B20139
:101B3000B301B401B501B601B701B801B901BA01E9
:101B4000BB01BC01BD01BE01BF01C001C101C20199
:101B5000FF300313CC00D030831203178D00003008
:101B60008F008A11031309218A151F179F178316E7
:101B70009F1383121F14831603170908C0391F38D7
:101B8000890003131F129F12FF300317880083126E
:101B9000031394128316CC124C0887004C164C0881
:101BA0008700CC114C08870001308312940000306C
:101BB000831694000108C739083881008312900108
:101BC0000030F80006389200FF30831692004C1166
:101BD0004C08870083120711831609130C308312F7
:101BE000970083169B019C0101309D00CC104C088E
:101BF0008700831287100C309D000130800003178E
:101C00008701880189018316031397018A118312C2
:101C100057218A158A1161218A158A11BC298A15D2
:101C20008A11F8298A15013083160317C8005E301F
:101C3000C7000130CA002C30C9008A118312031377
:101C400070228A15D63003178D0000308F008A115C
:101C5000031309218A15023083160317C300FA30D3
:101C6000C8008A1183120313C0228A158316031732
:101C7000C30B2F2EDA3083128D0000308F008A11B3
:101C8000031309218A1528080F3C031C562E031D37
:101C90004D2E27089F3C031C562E83168910831255
:101CA000891083160910831209145E2E83160910F9
:101CB0008312091083168910831289142708403C67
:101CC000031D682E28081F3C031D682EA801A701CC
:101CD000A70A0319A80A831608178312081F882E5B
:101CE0008316891083128910831609108312091430
:101CF00083160317C801C830C7000130CA00F4308A
:101D0000C9008A118312031370228A150028862EB7
:101D1000831688178312881F422F83160910831297
:101D20000910831689108312891401308316031752
:101D3000C8002C30C7000130CA00F430C9008A1135
:101D40008312031370228A157508F6008A1108237E
:101D50008A158A1185238A158A11D4228A158A1137
:101D6000F5228A15F508031DB92E7608F500FC0A40
:101D7000BA2EFC017C08083C0318CA2E7D08633C7F
:101D8000031CC42E0130F5007E08633C031CCA2EE0
:101D90006330F5008A11DE2C8A158A112D2D8A15E3
:101DA0007508313C031CDC2E0310200DFF3C83160C
:101DB000CA00FF30CB0083127508323C031DE52EAC
:101DC000FF308316CA00CB0083127508323C03181B
:101DD000F32EFF308316CA0003108312200DFF3C40
:101DE0008316CB00831283164908323C0318062F52
:101DF000C80A89108312891083164808283C0318E2
:101E0000052F0310CA0C0310CB0C0B2FC80189102F
:101E10008312891483164908463C0318302F8A110F
:101E2000831257218A158A1161218A158316031797
:101E3000C8016430C700CA01C830C9008A118312C2
:101E4000031370228A158A11F5228A158316490810
:101E5000463C0318302F8A1183128A2D8A15831667
:101E60004A080317C7008A118312031379248A15BD
:101E700083164B080317C7008A1183120313972494
:081E80008A15A42E432E630015
:04400E00F52CFF3F4F
:00000001FF
